:1000000012C02CC02BC0B1C000C128C027C026C060
:10001000C2C724C023C022C021C020C048C01EC007
:100020001DC01CC01BC011241FBECFE5D4E0DEBF25
:10003000CDBF10E0A0E6B0E0ECEDFAE102C0059023
:100040000D92A23AB107D9F721E0A2EAB0E001C0CF
:100050001D92AE3BB207E1F771D93ECDD1CFDC01A5
:10006000CB016FB7F89448B3416058B35E7F37E077
:100070002D9148BB220F30F058BB000027FB3150B8
:1000800031F0F7CF000027FB315058BB91F737E034
:1000900048BB3EF0000058BB2D91019751F76FBF50
:1000A00008952D91019758BB21F76FBF08951F92B6
:1000B0000F920FB60F9211248F9385B18093A200F7
:1000C0008F910F900FBE0F901F90189587B1866685
:1000D00087B986B18F6E86B908958091A200089580
:1000E00081B38C7F81BB82B3876082BB08951092FD
:1000F000A30080990EC080916000882331F081E0D8
:100100008093A3001092600007C084E08093A30056
:1001100003C081E08093600082990EC080916100ED
:10012000882331F082E08093A3001092610007C021
:1001300085E08093A30003C081E0809361008199F2
:100140000EC080916200882331F083E08093A30089
:100150001092620007C086E08093A30003C081E094
:10016000809362008091A30008951F920F920FB6B2
:100170000F9211242F933F934F935F936F937F932D
:100180008F939F93AF93BF93EF93FF938091A400BE
:1001900090E0FC01EE0FFF1FEE0FFF1F8E0F9F1F61
:1001A000FC01E05AFE4FE181F0E0E956FF4F80810B
:1001B00088BB81E090E00090A40002C0880F991FE6
:1001C0000A94E2F785BB8091A4008F5F863019F016
:1001D0008093A40002C01092A4008091AC008823F8
:1001E00019F0E3D41092AC00FF91EF91BF91AF9161
:1001F0009F918F917F916F915F914F913F912F913F
:100200000F900FBE0F901F9018951F920F920FB670
:100210000F9211242F933F934F935F938F939F934C
:10022000AF93BF93EF93FF9315BA8091A50081110F
:1002300099C08091A40090E0FC01EE0FFF1FEE0F2B
:10024000FF1F8E0F9F1FFC01E05AFE4F828183BD6E
:100250008091A40090E0FC01EA55FF4F208121111C
:100260000DC0FC01EE0FFF1FEE0FFF1FE80FF91F7F
:10027000E05AFE4F2381222309F45AC0FC01EE0FFD
:10028000FF1FEE0FFF1FE80FF91FE05AFE4F2481FA
:100290002F5F233061F0FC01EE0FFF1FEE0FFF1FF9
:1002A0008E0F9F1FFC01E05AFE4F2483E2C0FC0129
:1002B000EE0FFF1FEE0FFF1FE80FF91FE05AFE4F72
:1002C000148223812F5F2383293161F4FC01EE0F17
:1002D000FF1FEE0FFF1FE80FF91FE05AFE4F1382BA
:1002E00020E00DC02D3058F0FC01EE0FFF1FEE0F87
:1002F000FF1FE80FF91FE05AFE4F30813183FC01E8
:10030000EE0FFF1FEE0FFF1FE80FF91FE05AFE4F21
:1003100030E0A901440F551F240F351F220F331F52
:1003200026533F4FD901A80FB91F8C918283A1C0DA
:10033000FC01EE0FFF1FEE0FFF1FE80FF91FE05A41
:10034000FE4F20813181321709F493C0FC01EE0F7A
:10035000FF1FEE0FFF1F8E0F9F1FFC01E05AFE4F85
:10036000218387C0813009F084C08091A40090E08F
:10037000FC01EE0FFF1FEE0FFF1F8E0F9F1FFC01F2
:10038000E05AFE4F828183BD8091A40090E0FC0181
:10039000EE0FFF1FEE0FFF1FE80FF91FE05AFE4F91
:1003A0003081218123130DC0FC01EE0FFF1FEE0FE2
:1003B000FF1FE80FF91FE05AFE4F2381222309F4A3
:1003C00058C0FC01EE0FFF1FEE0FFF1FE80FF91FD3
:1003D000E05AFE4F24812F5F233061F0FC01EE0FC5
:1003E000FF1FEE0FFF1F8E0F9F1FFC01E05AFE4FF5
:1003F00024833FC0FC01EE0FFF1FEE0FFF1FE80F2D
:10040000F91FE05AFE4F148223812F5F2383293185
:1004100061F4FC01EE0FFF1FEE0FFF1FE80FF91F45
:10042000E05AFE4F138220E00CC02D3050F0FC014A
:10043000EE0FFF1FEE0FFF1FE80FF91FE05AFE4FF0
:100440003183FC01EE0FFF1FEE0FFF1FE80FF91FB6
:10045000E05AFE4F30E0A901440F551F240F351F0D
:10046000220F331F26533F4FD901A80FB91F8C917C
:100470008283FF91EF91BF91AF919F918F915F9197
:100480004F913F912F910F900FBE0F901F90189595
:10049000DC01E0E6F1E02EE731E08AE09D91943660
:1004A00010F0808301C090833596E217F307B1F70F
:1004B0000895DC01E0E6F1E04EE751E06DEC3AE052
:1004C0009C91943618F03083358315C0969F912DFA
:1004D000112496959695969590839C91969F812D43
:1004E0001124869586958695880F282F220F220F36
:1004F000820F981B958311963A96E417F50701F73A
:1005000008958093A50008952F923F924F925F9295
:100510006F927F928F929F92AF92BF92CF92DF9213
:10052000EF92FF920F931F93CF93DF938A3008F4DB
:100530008AE00F2EF0E6AF2EF1E0BF2EF02D0F2E49
:10054000FAEC8F2EF0E09F2EF02D0F2EF7E9CF2E34
:10055000F0E0DF2EF02D382E3094E82EF12C412CD7
:10056000512C32014A94232C22C0F80181918F0131
:100570008E9DB0018F9D700D1124072E000C880BED
:10058000990BA301920151DA230D288326960C15AD
:100590001D0559F7F5012282F5E0AF0EB11C8FEF72
:1005A000881A980AEEE7AE16E1E0BE0621F00EE7E3
:1005B00010E0E401DACFDF91CF911F910F91FF900E
:1005C000EF90DF90CF90BF90AF909F908F907F90F3
:1005D0006F905F904F903F902F900895843608F071
:1005E00083E6682F70E0762F6627072E000C880BB5
:1005F000990B24E630E040E050E017DA822F84DFE8
:10060000089584E6EBDF87B38C6387BB84B38F6385
:1006100084BB85B5846085BD89B7806C89BF08952A
:100620002F923F924F925F926F927F928F929F9202
:10063000AF92BF92CF92DF92EF92FF920F931F93F0
:10064000CF93DF9300D000D0CDB7DEB74C0180E66A
:1006500091E09A8389830F2EFAECAF2EF0E0BF2E43
:10066000F02D0F2EFAE02F2EF02D412C512C3201BF
:100670004A947401F40180818A3088F520822FC069
:10068000F80161918F01F7013080639DB001112461
:10069000072E000C880B990BA3019201C6D9309448
:1006A000320EEB81FC8130823696FC83EB83EC15B5
:1006B000FD0531F7FFEF8F1A9F0AF70180818095C2
:1006C000E981FA8182833596FA83E983FFEFAF1AD5
:1006D000BF0A80EDA81680E0B80659F609C00EE7FB
:1006E00010E0650196E9C90ED11CBC82AB82C8CF6F
:1006F0000F900F900F900F90DF91CF911F910F915E
:10070000FF90EF90DF90CF90BF90AF909F908F9031
:100710007F906F905F904F903F902F9008957F92C1
:100720008F929F92AF92BF92CF92DF92EF92FF9201
:100730000F931F93CF93DF9300D000D000D0CDB79D
:10074000DEB77C018E010F5F1F4F6E0187E0C80E80
:10075000D11C0F2EF3E67F2EF02D0F2EF4E68F2EF8
:10076000912CA12CB12CF02DF70181917F018436C1
:1007700018F4F801808302C0F8017082F8016081EA
:1007800070E0762F6627072E000C880B990BA501C9
:1007900094014BD9F80121938F01EC15FD0521F748
:1007A000CE0101963DDF26960FB6F894DEBF0FBE50
:1007B000CDBFDF91CF911F910F91FF90EF90DF9010
:1007C000CF90BF90AF909F908F907F900895DC0165
:1007D000E6EAF0E02CEA30E08D918193E217F3072E
:1007E000D9F70895E0E6F1E08AE080838583828787
:1007F0008787848B818F089581E08093AC00089572
:10080000282F207730E0A901440F551F220F331FF6
:10081000220F331F220F331F240F351F35952795C5
:100820003595279535952795359527958F70820FA6
:10083000089540E050E060E07DEC879F312D112469
:10084000232F269526952695220F922F990F990FE3
:10085000290F821B282F832F86958695869530E059
:10086000042E02C0220F331F0A94E2F7622B4C5F62
:100870005F4F4031510509F7862F0895CF93C82F58
:10088000C2716111C0644111C068CDD080EDF7D054
:100890008EE0F5D08C2FF3D096D0CF910895EF92C3
:1008A000FF920F931F93CF93DF93EC018B017A019B
:1008B000BAD080EDE4D080E0E2D0C2D081EDDFD0CC
:1008C00080E007D19DDFF701808380E002D198DFCF
:1008D000F801808381E0FDD093DF888374D0DF91BD
:1008E000CF911F910F91FF90EF9008951F93CF9399
:1008F000DF93C82FD62F142F96D080EDC0D080E084
:10090000BED0812F96DFBBD08D2F93DFB8D08C2F38
:1009100090DFB5D058D0DF91CF911F910895EF921D
:10092000FF920F931F93CF93DF937C018B01EA011A
:100930007AD080EDA4D084E0A2D082D081ED9FD087
:1009400080E0C7D05DDFF701808380E0C2D058DF50
:10095000F801808381E0BDD053DF888334D0DF91FC
:10096000CF911F910F91FF90EF9008951F93CF9318
:10097000DF93182FD62FC42F56D080ED80D084E07F
:100980007ED0812F56DF7BD08D2F53DF78D08C2FF8
:1009900050DF75D018D0DF91CF911F9108958B98BB
:1009A000939A10927F01089580917F0190B398707F
:1009B00090937F01811105C081E0911103C080E017
:1009C000089580E008958F9A979883E397E00197C0
:1009D000F1F78E9A9698E3E3F7E03197F1F78F9865
:1009E000979A83E397E00197F1F78E98969AE3E35D
:1009F000F7E03197F1F7869902C082E001C080E00C
:100A0000879B8160E3E3F7E03197F1F7E3E3F7E0F9
:100A10003197F1F7E3E3F7E03197F1F7E3E3F7E03C
:100A20003197F1F708958E9A969883E397E00197AE
:100A3000F1F78F9A979883E397E00197F1F708957C
:100A40008E98969A83E397E00197F1F78F98979A9B
:100A500083E397E00197F1F78E9A969883E397E006
:100A60000197F1F78F9A979883E397E00197F1F751
:100A700008958E98969A8F98979AA5DF089598E092
:100A800088231CF08E9A969802C08E98969AE3E37B
:100A9000F7E03197F1F78F98979AE3E3F7E0319712
:100AA000F1F78F9A9798880F915051F78E98969AF0
:100AB00083E397E00197F1F78F98979AE3E3F7E0E4
:100AC0003197F1F780B38F9A979886FB882780F942
:100AD0000895282F8E98969A98E080E0880F8F9836
:100AE000979AE3E3F7E03197F1F7869981608F9A5F
:100AF0009798E3E3F7E03197F1F7915079F72111F7
:100B000003C08E9A969802C08E98969AE3E3F7E017
:100B10003197F1F78F98979AE3E3F7E03197F1F780
:100B20008F9A9798E3E3F7E03197F1F78E98969ACA
:100B30000895FC019081242F30E0D901A90FB11D47
:100B4000AF3FB10509F02CF4940F90839F3F79F4E7
:100B500002C08FEF8083FB015081852F90E0821BC4
:100B6000930B1AF0541B50830895FB0110820895D3
:100B70008095853564F4982F990F890F982F90955B
:100B8000FB019083F9011082FA0180830895FB0133
:100B900010828555982F990F890FF9018083FA01EA
:100BA00080830895B89AC098089562E170E082E960
:100BB00091E055DA0895CF92DF92EF92FF920F9372
:100BC0001F93CF93DF93362F90E0FC01EE0FFF1FB2
:100BD000E80FF91FC0916400D0E08F010E561E4F40
:100BE0004C9FC0014D9F900D11240F2EF3E6EF2E68
:100BF000F12CF02DB70106D7D8016C938F010F5F50
:100C00001F4FDF01A058BE4F4C93C8018E569E4F18
:100C10006C013C9FC0013D9F900D1124B701F2D69D
:100C2000D6016C933296D801A058BE4F3C938F01E9
:100C30000E561E4F2C9FC0012D9F900D1124B70101
:100C4000E1D6D8016C93E058FE4F2083DF91CF911D
:100C50001F910F91FF90EF90DF90CF900895FB01CF
:100C6000228141816081A7DF08950F931F93CF9365
:100C7000DF93082F162FD42FC0E02D2F412F602F88
:100C80008C2F99DFCF5FC630C1F7DF91CF911F91D5
:100C90000F910895CF93C0E020E040E060E08C2FFA
:100CA0008ADFCF5FC630C1F7A7DDCF910895CF921D
:100CB000DF92FF920F931F93CF93DF9300D01F9289
:100CC000CDB7DEB70091B4001091B5000F3F11050C
:100CD00009F0C0F5F090B30082E08F1538F1CF2C09
:100CE000D12C86E0C816D1049CF11CC00D5F1F4FAB
:100CF0009801A1E8B0E8BBD6880F892F881F990B0F
:100D000091959E012D5F3F4FAE014E5F5F4FBE013B
:100D10006F5F7F4F800F2CDF2B814A81698183E0D9
:100D20008F0D49DFF394F092B30002C01092B3002C
:100D30008091B4009091B50001969093B500809396
:100D4000B40004C01092B5001092B40055DD22C06A
:100D50009801A1E8B0E88BD6880F892F881F990BDE
:100D600091959E012D5F3F4FAE014E5F5F4FBE01DB
:100D70006F5F7F4F800FFCDE2B814A8169818F2D51
:100D80001ADF83E0C80ED11C86E0C816D1040CF42B
:100D9000ADCFC8CF0F900F900F90DF91CF911F91E3
:100DA0000F91FF90DF90CF900895CF92DF92EF9256
:100DB000FF921F93CF93DF9300D01F92CDB7DEB782
:100DC000C090B100D090B200C11485E0D80638F5CB
:100DD00010E0E12CF12C9701ABEABAEA48D69695DF
:100DE0008795969587959E012D5F3F4FAE014E5F8B
:100DF0005F4FBE016F5F7F4F8C0DBADE2B814A8142
:100E00006981812FD8DEF3941F5F163021F78FEFB1
:100E1000C81AD80AD092B200C092B10004C0109291
:100E2000B2001092B100E8DC0F900F900F90DF91AC
:100E3000CF911F91FF90EF90DF90CF900895EF92A8
:100E4000FF921F93CF93DF9300D01F92CDB7DEB7F1
:100E5000E090AF00F090B0008FEFE816F10409F0D9
:100E6000E8F410E09E012D5F3F4FAE014E5F5F4FF3
:100E7000BE016F5F7F4F812F8E0D7ADE2B814A81FD
:100E80006981812F98DE1F5F163061F78FEFE81AB6
:100E9000F80AF092B000E092AF0004C01092B000E7
:100EA0001092AF00A9DC0F900F900F90DF91CF91BF
:100EB0001F91FF90EF900895CF93C82F61111FC02D
:100EC0008091AE00811106C04C2F63E670E08DEA80
:100ED00090E02FDE80916300811106C04C2F6DEAF7
:100EE00070E08EEA90E025DE8091AD00811133C084
:100EF0004C2F6EEA70E083E690E01BDE2CC0809100
:100F0000AE00811106C04C2F6DEA70E083E690E0E0
:100F100010DE80916300811106C04C2F6EEA70E0F4
:100F20008DEA90E006DE8091AD00811114C04C2F57
:100F300063E670E08EEA90E0FCDD0DC02091AE002B
:100F40004091AD00609163008C2F35DECF5FC630DD
:100F5000A9F752DC02C0C0E0F1CFCF9108958436EA
:100F600018F480936400089583E6809364000895E4
:100F700090E0FC01EE0FFF1F8E0F9F1FFC01E05859
:100F8000FE4F8081DA018C938181DB018C93828119
:100F9000F901808308951F920F920FB60F921124CA
:100FA0002F933F934F935F936F937F938F939F9371
:100FB000AF93BF93EF93FF9380E090E051E04FEF4A
:100FC0009C01FC01EE0FFF1FE80FF91FE654FF4FD5
:100FD00060816F3F41F1FC01EE0FFF1FE80FF91F29
:100FE000E654FF4F61817281672B79F0FC01EE0FAF
:100FF000FF1F2E0F3F1FF901E654FF4F2181328161
:1010000021503109328321830EC0FC01EE0FFF1FF6
:101010002E0F3F1FF901E654FF4FA081B0E0AC5501
:10102000BE4F5C93408301968530910549F687EF6A
:101030009FEF9DBD8CBDFF91EF91BF91AF919F91AF
:101040008F917F916F915F914F913F912F910F9071
:101050000FBE0F901F9018959091BA00891771F0EC
:1010600021E030E0A901F901EE0FFF1FE20FF31FAD
:10107000E654FF4F908198130EC002C040E050E04C
:10108000FA01EE0FFF1F4E0F5F1FFA01E654FF4FEC
:101090007283618308952F5F3F4F2530310511F72B
:1010A0009091BA009F3F71F021E030E0A901F90171
:1010B000EE0FFF1FE20FF31FE654FF4F90819F3F9B
:1010C00079F402C040E050E0FA01EE0FFF1F4E0F2E
:1010D0005F1FFA01E654FF4F808372836183089596
:1010E0002F5F3F4F2530310509F70895CF93DF93E8
:1010F0001092A4018091B6009091B7000196909350
:10110000B7008093B600883E934098F04BEA51E0D8
:101110006AEA71E089EA91E002DC8091B600909180
:10112000B7008C3F934058F11092B7001092B60070
:1011300026C03ADC882319F14BEA51E06AEA71E0F3
:1011400089EA91E0ACDBC9D7C82FD0E0CC0FDD1F16
:10115000CF3FD10519F010F0CFEFD0E084E68C9F9F
:1011600090018D9F300D1124A1E8B0E880D4880F44
:10117000892F881F990B9195F2DE8C2FC5D989EAAA
:1011800091E097D96AE070E080E066DFDF91CF916F
:1011900008951092A5018091AC01811103C0A7D7D9
:1011A0008093AC018091AC01823011F01092AC01BF
:1011B00061E070E081E050DF08951092A60185E0C3
:1011C00090E075D4823079F028F4882341F08130A2
:1011D00041F010C0833049F0843049F00BC05ADD33
:1011E00009C065DD07C0E1DD05C029DE03C060E0A0
:1011F0008AE062DE64E670E082E02EDF08951092FD
:10120000A7018091AC01823019F4ACD01092AC01EE
:1012100064E670E083E020DF0895CF93DF9389E0F8
:1012200090E045D49CDE87E090E041D4D7D985E0BA
:1012300090E03DD48093B90084E090E038D480936E
:10124000B80082E090E033D4D82F81E090E02FD432
:10125000C82F80E090E02BD44D2F6C2F06DDCCDA28
:1012600083E090E024D4882319F081E04AD902C0B9
:1012700080E047D9DF91CF910895EAEBF0E08FEF5E
:10128000808383838683818784871FBC8EB5856036
:101290008EBD87EF9FEF9DBD8CBD89B7846089BFF0
:1012A00061E070E080E0D8DE61E070E081E0D4DEF3
:1012B00064E670E082E0D0DE64E670E083E0CCDEDD
:1012C000A0D9D7DB41E061E080E0D8DA68DB08D75D
:1012D00069DCFCD68AE090E0EAD38F3F61F560E0FC
:1012E00080E090E0ECD360E081E090E0E8D360E063
:1012F00082E090E0E4D363E689E090E0E0D365E04B
:1013000088E090E0DCD363E687E090E0D8D36AE041
:1013100086E090E0D4D364E085E090E0D0D360E054
:1013200084E090E0CCD361E083E090E0C8D360E05B
:101330008AE090E0C4D371DF789408959EDFC4EA18
:10134000D1E088818111D2DE8981811122DF8A81F9
:10135000811133DF8B81811152DF8AE18A95F1F7A8
:1013600000C0EFCF2F923F924F925F926F927F9289
:101370008F929F92AF92BF92CF92DF92EF92FF92A5
:101380000F931F93CF93DF93CDB7DEB766970FB65A
:10139000F894DEBF0FBECDBF86E0E8E6F0E0DE01E8
:1013A000119601900D928A95E1F72BEB31E04AEB13
:1013B00051E069EB71E080E0DBDD0F2EF9EBEF2E01
:1013C000F1E0FF2EF02D00E010E00F2EFCEBCF2E11
:1013D000F1E0DF2EF02DF70161917F01C8016FD39D
:1013E0000F5F1F4FEC14FD04B1F7512C0F2EFDEAD7
:1013F000EF2EF1E0FF2EF02D332433940F2EF3EB7C
:10140000CF2EF1E0DF2EF02DED8AFE8A87E090E00E
:101410004ED38093BC01A3DD9091BC018DEC989FCD
:10142000812D1124869586958093BD01F7019083C7
:10143000E3EBF1E03082EEEAF1E0A4EBB1E081937E
:101440001D92EC15FD05D9F7C70169D980E059D87F
:10145000CE0101961DD8FFEF20E782E0F150204039
:101460008040E1F700C0000083EB91E0B0D912DCCE
:1014700065E670E080E0F3DBBFD9BED910E06BC059
:10148000813029F0843071F598EC951548F5812F5D
:1014900090E0FC01E355FE4F2091BD012083FC014B
:1014A000ED54FE4F10821F5F163009F410E0812FBB
:1014B00090E0FC01E355FE4F2091BC012083FC012C
:1014C000ED54FE4F3082C7012AD983EB91E07FD9DA
:1014D000E1DB65E670E0812FC2DB8ED9512C02C0C2
:1014E000539433C08091C900833029F0863069F568
:1014F000E8ECE51548F5812F90E0FC01E355FE4F3F
:101500002091BD012083FC01ED54FE4F108211504B
:10151000173008F015E0812F90E0FC01E355FE4FF5
:101520002091BC012083FC01ED54FE4F3082C701A5
:10153000F6D883EB91E04BD9ADDB65E670E0812F07
:101540008EDB5AD9512C01C053948FEC97E0019750
:10155000F1F700C00000CBD58093C900823009F0BC
:101560008FCFE12FF0E0ED54FE4F108283EB91E03E
:101570002ED9113009F489C120F0153009F415C2B3
:1015800016C285E0EEE6F0E0DE011D9601900D92B8
:101590008A95E1F785E0E3E7F0E0DE011796019038
:1015A0000D928A95E1F71ED987E090E080D2809372
:1015B000BC01982F9695969596959093BD01F7014D
:1015C00080838183E3EBF1E010821092B401F70194
:1015D00092831092B50193831092B6019483109276
:1015E000B70195831092B80180E08BD74BEA51E0A8
:1015F0006AEA71E089EA91E052D989EA91E059D723
:10160000C7018DD8FFEF20E782E0F15020408040F5
:10161000E1F700C0000083EB91E0D9D83BDB65E641
:1016200070E080E01CDB65E670E0832D18DBE4D819
:1016300010E000E00F2EF4E12F2EF02D58D580930E
:10164000C900B2D9882361F0023050F44BEA51E06E
:10165000BE016E5E7F4FCB0122D989EA91E029D786
:101660008091C900813021F08430B9F5173998F1A3
:10167000043009F100FBAA24A0F8B12CF501E755CC
:10168000FE4F80818F5F8083202F30E0EDE0F0E01F
:10169000EC0FFD1FE20FF31F90819817B8F4E7E0FD
:1016A000F0E0EC0FFD1FE20FF31F8081F501E7551D
:1016B000FE4F80830BC0E9EAF1E082818F5F828375
:1016C0009989981718F48B858093AB0189EA91E08A
:1016D000F0D610E0D0C01F5FCEC0833031F086302E
:1016E00009F045C0173908F440C0043079F100FB17
:1016F000662460F8712CF301E755FE4F808181501C
:101700008083202F30E0EDE0F0E0EC0FFD1FE20FD2
:10171000F31F9081981720F4F301E755FE4F908353
:101720008EEF800F8230E0F4A7E0B0E0AC0FBD1F79
:10173000A20FB31FF301E755FE4F40818C9148176C
:1017400078F4F301E755FE4F90830AC0E9EAF1E02F
:101750008281815082839989981710F49093AB010C
:1017600089EA91E0A6D610E086C01F5F84C082306F
:1017700009F081C00F5F023039F4E9EAF1E04281FB
:1017800061818081B3D81FC0043039F4E9EAF1E007
:10179000428161818081EAD822C00530A1F40F2EF8
:1017A000F9EA8F2EF1E09F2EF02DF40142804BEAF2
:1017B00051E06AEA71E0C401B2D8442DF4016181BC
:1017C0008081D4D813C00230A0F0023041F44BEA3B
:1017D00051E06AEA71E089EA91E0A1D807C00430DB
:1017E00029F4E9EAF1E024E62083218289EA91E004
:1017F00060D650DA8091BD01F701808381838283B6
:101800008383848385830430C9F0F02FF1709F2E89
:101810008F2E880C65E670E0882D21DA65E670E091
:1018200081E0880D1CDAE92DF0E0EE0FFF1F8091BA
:10183000BC01E355FE4F8083818316C08FEA91E09F
:101840009C8B8B8B6894992491F865E670E0892DC8
:1018500006DA8091BC01EB89FC898193FC8BEB8BD0
:101860009394F6E09F12F1CFC7D78D899E8957D701
:1018700083EB91E0ACD78FEC97E00197F1F700C0D4
:101880000000053009F0DACEC1CD85E090E00FD13F
:10189000082F00DA89E090E00AD161DB10E065E60C
:1018A00070E0812FDCD91F5F1630C9F7A5D73092C1
:1018B000B801E3EBF1E010821092B4011092B5018F
:1018C0001092B6011092B701CF0181D786E0E8E708
:1018D000F0E0DE01179601900D928A95E1F787E01E
:1018E00090E0E5D07BD60C87CE010796D1D5912C20
:1018F00010E0FDD38093C9001F5F123310F1023056
:1019000079F028F4002341F0013041F019C0033090
:1019100049F0043049F014C0BDD950C0C8D94EC0F8
:1019200044DA4CC08CDA4AC060E08AE0C5DA8091C3
:10193000C900823021F18330B1F0813049F50CC00B
:1019400010E08230F9F0833089F0813021F50F5FAB
:10195000053021F400E002C010E000E00C87CE0169
:10196000079696D518C010E001C010E00150053070
:1019700008F004E00C87CE0107968AD50CC010E071
:1019800001C010E09394602F85E090E098D003C0F0
:1019900010E001C010E08FEC97E00197F1F700C074
:1019A000000091E09912A5CF31CD1CD710C01530A1
:1019B00009F02CCD0CC00F5F10E0D0CF8091C90092
:1019C0008230F9F2833089F2813021F7F4CF25DCBF
:1019D00081E066960FB6F894DEBF0FBECDBFDF91F3
:1019E000CF911F910F91FF90EF90DF90CF90BF901C
:1019F000AF909F908F907F906F905F904F903F90AF
:101A00002F90089597FB072E16F4009406D077FDCB
:101A100008D039D007FC05D03EF4909581959F4FB2
:101A20000895709561957F4F0895A1E21A2EAA1B23
:101A3000BB1BFD010DC0AA1FBB1FEE1FFF1FA2177E
:101A4000B307E407F50720F0A21BB30BE40BF50B7B
:101A5000661F771F881F991F1A9469F76095709504
:101A6000809590959B01AC01BD01CF010895A29F87
:101A7000B001B39FC001A39F01D0B29F700D811D23
:101A80001124911D0895AA1BBB1B51E107C0AA1F79
:101A9000BB1FA617B70710F0A61BB70B881F991F0F
:101AA0005A95A9F780959095BC01CD010895E199CB
:101AB000FECF9FBB8EBBE09A99278DB30895262F4A
:101AC000E199FECF9FBB8EBB2DBB0FB6F894E29A77
:0C1AD000E19A0FBE01960895F894FFCF34
:101ADC00010101FF63FF0000010203040506173B2F
:101AEC001F0C6300000101006464646464640128D9
:101AFC00465A7896AABED2E6F0FAFAFAF0E6D2BEC8
:101B0C00AA96785A4628010004080C1014181C20B8
:021B1C00247C27
:00000001FF
